S3152000F00039F1002057F10020F1F0002070B50546B7
S3152000F0104FF43026304600F059F8042811D1094C17
S3152000F020206940F0020020616561206940F04000BF
S3152000F0302061304600F04AF8216941F6FD72114000
S3152000F040216170BD0020024008490420CA68D20709
S3152000F05001D001207047CA68520701D502207047A7
S3152000F060C968C906FBD5032070470000002002406E
S3152000F0700248016941F08001016170470020024089
S3152000F080F0B506464FF400570D46384600F01EF8F8
S3152000F09004280CD1064C206940F0010020613580FF
S3152000F0A0384600F013F82169BA1E11402161F0BDDF
S3152000F0B000200240034802494160034941607047ED
S3152000F0C02301674500200240AB89EFCD00B50346FA
S3152000F0D0FFF7BAFF03E000BFFFF7B6FF5B1E01286C
S3152000F0E003D0002B00D1052000BD002BF4D1FAE778
S3152000F0F0F0B50E4604004FF0000708D03EB172B6B8
S3152000F100FFF7D8FF0B493520C86000250BE001200A
S3152000F110F0BD2046FFF77AFF042801D0012704E03E
S3152000F12004F500646D1CB542F3D3FFF7A1FF62B668
S3152000F1303846F0BD0020024030B50446002041B1DB
S3152000F1403AB1002302E0E55CCD545B1C9342FAD32E
S3152000F15030BD012030BD2DE9F0414FF000081546A5
S3152000F1600E460700444605D025B11EB172B6FFF7FC
S3152000F170A1FF0FE00120BDE8F08106EB44000188E5
S3152000F18007EB4400FFF77CFF042802D04FF001086C
S3152000F19003E0641CB4EB550FEFD3FFF769FF62B6AB
S3092000F1A04046E8E7F0
S70500000000FA
